:10000000F128FF3FFF3FFF3FFF00030E8301B200D7
:100010000408B1000A08B3008A017108BA00700828
:10002000B90001300C05F1007108031930280C10DB
:10003000D8308F00F8308E00A00A2008643A031DE3
:100040003028A001A1032108FF3A031D30283B30CE
:10005000A100A2032208FF3A031D30283B30A20072
:1000600000308C180130F1007108031957288C10EA
:100070000F3085042330F000270870078400000843
:1000800086002809F00070088505A70A2808F100F5
:10009000F10D71107108A8007108083C031852286E
:1000A0000130A8002708033C03185728A7013A0885
:1000B000F1003908F00033088A0031088400320E5C
:1000C0008300FF0E7F0E090064000D3003138312BE
:1000D000FB00FF30FA00FB0B6E287128FA0B6E282C
:1000E0006B28F330FA00FA0B7328000008000313A2
:1000F0008312B8010030051A0130F1007108003A8E
:10010000031D992864200030051A0130F1007108A0
:10011000003A031D99280517381464200513003090
:10012000051A0130F1007108003A031D9928642076
:100130008F280030851A0130F1007108003A031D44
:10014000B82864200030851A0130F1007108003AA7
:10015000031DB8280517B814642005130030851A4C
:100160000130F1007108003A031DB8286420AE2860
:100170003808F000080003138312A0012908A10029
:100180002A08A2000800C034F934A434B0349934E9
:1001900092348234F834803490340800031383128C
:1001A000F8010830FC00700DF80D7408F80203180F
:1001B000DB28F8070310F00DFC0BD328080003130D
:1001C00083122D088A002B088200080040347934FD
:1001D0002434303419341234023478340034103476
:1001E00008000730031383129F000E30831681002E
:1001F0008312850186013030831685008601033025
:100200008C0083128C01D8308F00F8308E000130C2
:100210009000FF30831692000D3083129200C030A0
:100220008B00A7010130A800A201A101A0010530A7
:10023000AA00A901AE01A301A401A501A601643091
:10024000AF002F08003A03192829AF0364202129A1
:10025000640077207008B0002E08003A031DDF29E3
:100260003008013A031D48292A08003CFF300318D2
:100270000030F2002908003CFF3003180030F00085
:100280007208F004031948298517BB200130AE001D
:100290003008023A031D6E290F302907F200720858
:1002A000A90072083B3C03185C29A901AA0A2A0884
:1002B0003B3C03185C29AA012A080A3AFF30031DB7
:1002C0000030F2002908003CFF3003180030F00035
:1002D0007208F00503196E29AA01A901C330B600FE
:1002E0000030B7000A30F4002A08F000CE200030B9
:1002F000F1003608F00737080318013FF1077008CE
:10030000AB007108AD000A08AC00DF20F0002C083B
:100310008A007008A300E630B4000030B5000A304F
:10032000F4002A08F000CE207808F0000030F10038
:100330003408F00735080318013FF1077008AB00D7
:100340007108AD000A08AC00DF20F0002C088A001C
:100350007008A4000A30F4002908F000CE20003014
:10036000F1003608F00737080318013FF10770085D
:10037000AB007108AD000A08AC00DF20F0002C08CB
:100380008A007008A5000A30F4002908F000CE2089
:100390007808F0000030F1003608F007370803183D
:1003A000013FF1077008AB007108AD000A08AC000E
:1003B000DF20F0002C088A007008A6007C2B2E0895
:1003C000013A031D8E2A3008013A031DEA29BB2099
:1003D0000230AE003008023A031D102A0F30290700
:1003E000F2007208A90072083B3C0318FE29A9011B
:1003F000AA0A2A083B3C0318FE29AA012A080A3A3D
:10040000FF30031D0030F2002908003CFF300318C4
:100410000030F0007208F0050319102AAA01A901A2
:100420003230200203181D2A8930A3008630A40030
:100430008830A500CE30A6008D2AC330B60000302B
:10044000B7000A30F4002A08F000CE200030F10096
:100450003608F00737080318013FF1077008AB00B2
:100460007108AD000A08AC00DF20F0002C088A00FB
:100470007008A300E630B4000030B5000A30F40084
:100480002A08F000CE207808F0000030F10034088F
:10049000F00735080318013FF1077008AB00710839
:1004A000AD000A08AC00DF20F0002C088A007008BC
:1004B000A4000A30F4002908F000CE200030F1003A
:1004C0003608F00737080318013FF1077008AB0042
:1004D0007108AD000A08AC00DF20F0002C088A008B
:1004E0007008A5000A30F4002908F000CE20780832
:1004F000F0000030F1003608F00737080318013F1C
:10050000F1077008AB007108AD000A08AC00DF20ED
:10051000F0002C088A007008A6007C2B2E08023AF6
:10052000031D7C2B3008013A031D9A2A3F308505B4
:10053000BB20AE013230200203180F2BC330B600AF
:100540000030B7000A30F4002208F000CE2000305E
:10055000F1003608F00737080318013FF10770086B
:10056000AB007108AD000A08AC00DF20F0002C08D9
:100570008A007008A300E630B4000030B5000A30ED
:10058000F4002208F000CE207808F0000030F100DE
:100590003408F00735080318013FF1077008AB0075
:1005A0007108AD000A08AC00DF20F0002C088A00BA
:1005B0007008A4000A30F4002108F000CE200030BA
:1005C000F1003608F00737080318013FF1077008FB
:1005D000AB007108AD000A08AC00DF20F0002C0869
:1005E0008A007008A5000A30F4002108F000CE202F
:1005F0007808F0000030F1003608F00737080318DB
:10060000013FF1077008AB007108AD000A08AC00AB
:10061000DF20F0002C088A007008A6007B2BC33076
:10062000B4000030B5000A30F4002208F000CE20FB
:100630000030F1003408F00735080318013FF107D6
:100640007008AB007108AD000A08AC00DF20F000B4
:100650002C088A007008A3000A30F4002208F00079
:10066000CE207808F0000030F1003408F00735089B
:100670000318013FF1077008AB007108AD000A08CC
:10068000AC00DF20F0002C088A007008A4000A30BB
:10069000F4002108F000CE200030F1003408F0070B
:1006A00035080318013FF1077008AB007108AD0071
:1006B0000A08AC00DF20F0002C088A007008A500B2
:1006C0000A30F4002108F000CE207808F000003055
:1006D000F1003408F00735080318013FF1077008EE
:1006E000AB007108AD000A08AC00DF20F0002C0858
:1006F0008A007008A6007C2B2E08023A031DC32B2B
:100700002108003AFF30031D0030F2002208003AB1
:10071000FF30031D0030F0007208F0050319C32BF1
:1007200005177F308505AE01B0013008003A031D82
:10073000C12B77207008B0006420323020020318EB
:10074000AA2BA130A300A330A400AB30A5008630B3
:10075000A600B22BFF30A300FF30A400FF30A5009D
:10076000FF30A6002008003A031DC02B0030051BF7
:100770000130F20072080319BF2B0513C02B0517B7
:10078000952B3F30850564202829C52BFF3FFF3F6F
:02400E00103F61
:00000001FF
